:020000040800F2
:10000000501D0020CD000008F50F0008ED0E00087F
:1000100000000000000000000000000000000000E0
:10002000000000000000000000000000FF0F0008BA
:100030000000000000000000A5300008113F00088B
:10004000DF00000800000000DF000008DF000008FB
:10005000DF000008DF000008DF000008DF00000804
:1000600000000000DF000008A104000849050008A6
:10007000DF000008DF000008DF00000800000000CB
:10008000DF0000081D40000800000000DF0000083D
:10009000DF000008DF000008DF000008DF000008C4
:1000A000DF000008313A0008DF0000083540000892
:1000B000BD4000080348854600F0D6F800480047D8
:1000C000F9490008501D00200844F04704488047C3
:1000D00004480047FEE7FEE7FEE7FEE7FEE7FEE72F
:1000E000C13F0008B500000830B50B4601460020AE
:1000F0002022012409E00D46D5409D4205D31D462E
:100100009540491B2546954040191546521E002D25
:10011000F1DC30BD70B500242546002801DA012449
:100120004042002901DA01254942FFF7DDFFAC42D8
:1001300000D04042002C00D0494270BDF8B50024E8
:100140002546002904DA0E46012400214042B1412F
:10015000002B04DA1E46002352420125B34100F071
:1001600052F88C4617461E46AC4203D0002540424A
:100170008D41AC46002C02D0002657429E4161467C
:100180003A46334601B0F0BD10B5202A04DB0846DC
:10019000203AD040002110BD0B46D340D04020244F
:1001A000A21A91400843194610BD03460B439B0712
:1001B00003D009E008C9121F08C0042AFAD203E0DC
:1001C0000B780370401C491C521EF9D27047D2B202
:1001D00001E00270401C491EFBD270470022F6E786
:1001E00010B513460A4604461946FFF7F0FF2046AD
:1001F00010BD0321001D401E037812021A43491E40
:10020000F9D510467047F0B51FB40646002082B0FD
:1002100005464024019100901BE0019922460F46BB
:100220003046FFF7B1FF049A059B801A994110D31D
:1002300010461946224600F029F8361A8F410197D8
:10024000224601200021009F00F020F838184D417F
:1002500000902046641E0028DFDC019B00982946A0
:10026000324607B0F0BD0000064C0125064E05E001
:10027000E36807CC2B430C3C98471034B442F7D3C7
:10028000FFF71CFF205300084053000810B5202A38
:1002900004DB0146203A9140002010BD914020230C
:1002A0009C1A0346E3401943904010BDF0B51E4D23
:1002B000A8684007C00F34D1286C1D4C81B21B4880
:1002C0001C4B42690120D607002E02D09986204699
:1002D0001DE0944309D0184E164C96434034002E2E
:1002E0000ED0164E96430ED011E01987154B1448C8
:1002F000154A994201D2012100E00021116006E077
:100300002180124803E061801149498BD98741035C
:10031000490BA962A9680F4A1140091DA960034948
:1003200048610020F0BD00000024014000000020D2
:1003300000010020181300200000014000000244CA
:10034000000001C098080000C4000020000002C4A2
:10035000A0F7FF1FE8FFFF7FF0B51E4F85B03D6996
:100360001D4C6D1C3D61666AE46A029400966C4601
:1003700065800190218162810393386A01011748E9
:10038000091800220B4610461C5CFF2C04D1401CAF
:100390001028F9D3002A17D01022684600F01EF961
:1003A000386AF861401C38620001012109031030ED
:1003B000884201D900203862F8680949401CF86079
:1003C0004861002005B0F0BD1022684603F0E0FF50
:1003D000E6E70000A0000020AC52000800C00008C2
:1003E00018130020002911D08268521882604368D7
:1003F000934200DCD21A00238361C368934201D187
:100400000123436182600269521802610846704705
:10041000F0B50020174D0127144B154C3F03E86041
:1004200017E0625A144EB24212D1EA680919521CFE
:10043000EA604A882E69B24205D92A61E8614A68B1
:100440006A61421C2A624988994201D20B46A8611E
:10045000401C0101B942E4D3286A00011030B842BF
:1004600001D900202862E868F0BD0000FFC99A3B6E
:1004700000C00008A0000020AA55000010B504210B
:10048000054800F0CCF8054800218161C161016197
:10049000C1600162084610BD00C00008A000002035
:1004A00070B524490868401C0860234C2068800609
:1004B000C00F12D0214DA868E96B4018A860E96B05
:1004C00028466430064600F05DF820206060B06980
:1004D00000280AD00020E863E86020688005C00F8B
:1004E00002D001204002606070BD304600F086F905
:1004F00013494A78A3585B085B00A350F36832683D
:100500004E78D2180C4B0C33F2500B4B4A781B1D13
:10051000D658360C36040643D65049786258012323
:100520001A436250E8630749886880221043886054
:10053000D3E7000050000020000002400402002029
:1005400000530008003801400B480168491C016055
:100550000A4801688904C90F06D001214903416096
:1005600007490022CA63CA6001688903C90F02D023
:1005700001214904416070475400002000000240FE
:10058000A402002010B5002910D0C2684368521898
:10059000934200DCD21A00234361C2608468944213
:1005A00004D1012282618360C360C361084610BD2B
:1005B000FF2109220131D206002801D09162704743
:1005C0009161704701218902034A002801D091629C
:1005D000704791617047000000040048F0B585B095
:1005E00016460D46074600F075FA012002900020DD
:1005F0000090019503A9684600F0D4F9002476081C
:1006000007E060003A5A41190023012000F024FA63
:10061000641CA642F5D800F015FA05B0F0BD7FB510
:100620000D46044600F056FA00206A4631C203A97E
:10063000684600F0B7F900F005FA04B070BD00009C
:1006400006490020C861064801690422114301617E
:1006500001694022114301617047000030190020F8
:1006600000200240064A0021D16106490A6902239E
:100670001A430A61486108694022104308617047C3
:10068000301900200020024010B5054B0022DA612D
:10069000044A1369012423431361018010BD000043
:1006A000301900200020024010B50B4A0020D1680C
:1006B000CB060A4904D5C86902231843C861102033
:1006C000D3685B0705D5CB6901242343CB610421A3
:1006D0000843D06010BD0000002002403019002007
:1006E00070B5044600F008FA0546104E0AE0601C9A
:1006F00008D0002C04D000F0FFF9401BA04201D923
:10070000032070BDF068C007F1D1F068800601D504
:100710002020F060F068C00602D4F068400703D5DE
:10072000FFF7C2FF012070BD002070BD0020024015
:100730000A07120F01219140014201D001207047A8
:10074000002070470A07120F01219140014201D099
:100750000120704700207047FEB50B051B0E264C8C
:100760005B001C1909239B01E31801930F239B01D4
:10077000E31800930523DB01E618012307469B02DB
:100780000A07E5180020120F3B0003F03BFE0906A4
:100790000D11151A1F23272B2E00FF2924D8FF34F3
:1007A000FF340234A08E22E0FF291DD8019806E014
:1007B000FF2919D8019807E0802915D20098808A6E
:1007C00015E0802910D20098808E10E040290BD2CD
:1007D000B08A0CE0402907D2B08E08E0802903D20D
:1007E000A88A04E0802901D30020FEBDA88E11460E
:1007F000FFF79EFFFEBD0000980A0020C1688268D6
:10080000914201DA501A7047914202DC4269002A93
:1008100002D04068401A704780690028FBD0002051
:100820007047C2688168914201DA501A704791425C
:1008300002DC8269002A02D04068401A7047406991
:100840000028FBD000207047064901228969120365
:1008500008180101914201D3FF3801380249000113
:1008600040187047A000002000C0000800B510200C
:1008700000F092FD00BD0000F0B5364C4B001C1995
:1008800011239B01E518212302469B010020E31858
:10089000892A4AD011DC2F4F2F4E4B00DB199F19AC
:1008A0000F26B6019E19803A130003F0ABFD092014
:1008B000201522292D31353915008D2A45D00CDC23
:1008C0008A2A36D08B2A3BD08C2A05D140290CDAD3
:1008D0000B2080012018808AF0BD992A03D0A12A1C
:1008E00001D0FE2AF8D1802921DB0020F0BD084686
:1008F000F0BD1029F9DAFF34FF340234A08EF0BDC8
:100900001029F2DAB88AF0BD1029EEDAB88EF0BDFF
:100910000829EADAB08AF0BD0829E6DAB08EF0BD1F
:10092000FF29E2DC1420285EF0BDFF29DDDC988A77
:10093000F0BD8029D9DA012080022018808EF0BD18
:100940004029D2DA0D208001C4E74029CDDAA88AF7
:10095000F0BD0000980A00204002000010B5074AD0
:100960005068074B99695468A04201D05068996952
:10097000044A51430914401A10BD00002000002011
:1009800000E000E05505000031B500F0B5F8009C2E
:100990000546601C00D0641C00F0AEF8401BA0426D
:1009A000FAD338BDF8B5054623480F46017E012627
:1009B00001290BD0012101762868204C012807D09D
:1009C0002046FFF78DFE002813D030E00220F8BD4E
:1009D0002046FFF785FE002829D1FFF731FE20468B
:1009E000FFF77EFE06461648016904229143016125
:1009F0001DE00020C04338606C6812E02046FFF71D
:100A000031FE0E48FFF76CFE06460D4801690222D2
:100A100091430161002E01D03C6008E0012080027A
:100A20002418A868696880024018A042E6D80248E5
:100A3000002101763046F8BD3019002050C3000077
:100A40000020024003480169802211430161002017
:100A50007047000000200240F0B51FB405461A4858
:100A60000024017E16461F46012907D00121017688
:100A70001648FFF735FE002803D021E0022005B01C
:100A8000F0BD012D1AD0022D18D0042516E0220148
:100A900030463946FFF778FB81B2019862001018A2
:100AA000FFF7F2FD0948FFF71BFE09490A695208E2
:100AB00052000A61002803D1641CE4B2AC42E6D3C0
:100AC000014900220A76DAE73019002050C30000FD
:100AD0000020024005480169090605D50449416026
:100AE0000449416000207047012070470020024007
:100AF00023016745AB89EFCD0148006870470000CE
:100B00000001002002480168491C01607047000094
:100B10000001002010B50648016810221143016051
:100B2000002000F007F800F017F8002010BD0000CA
:100B30000020024010B5044600F040F97D21C900B4
:100B4000FFF7D2FA00F0B6F900222146501E00F05D
:100B500025F8002010BD000008B50F48816901226A
:100B600011438161816911400091C26901040A4306
:100B7000C261C0690022084000901146501F00F079
:100B80000DF800221146901E00F008F800221146D0
:100B9000501E00F003F808BD0010024010B502F02E
:100BA0005FFA10BDF8B504460068364DC00354D551
:100BB000E8690026C00007D4E86929040843E86111
:100BC000E8690840012600902F480168C90511D442
:100BD000014608688A1510430860FFF78DFF074635
:100BE00004E0FFF789FFC01B642823D8264800686B
:100BF000C005F6D5286A0321090208401FD06268A3
:100C00000A4082421BD0286A2A6A884301210904CB
:100C10000A432A622A6A8A432A622862C0070ED0DF
:100C2000FFF76AFF074607E0FFF766FFC11B17489B
:100C3000814201D90320F8BD286A8007F4D5286ACB
:100C4000032109028843616808432862002E04D00A
:100C5000E869012109078843E8612078C00705D0C9
:100C6000286BA168800880000843286320788006EC
:100C700005D5286B10218843E168084328630020CC
:100C8000F8BD000000100240007000408813000012
:100C9000F8B5044644480E460068C007C00FB0428D
:100CA0000AD241480168490849003143016000689F
:100CB000C007C00FB0425CD120783C4F800705D5FB
:100CC0007868F0218843A168084378602078C007DD
:100CD0003FD06068012813D03968022813D08907F3
:100CE000002946DA79688908890001437960FFF7AD
:100CF00003FF0546606801280DD0022817D024E0C4
:100D000039688903ECE78901EAE7FFF7F5FE411B43
:100D10002748814217D878680007800F0128F4D14E
:100D200017E0FFF7E9FE411B214881420BD87868A4
:100D30000007800F0228F4D10BE0FFF7DDFE411B16
:100D40001B48814201D90320F8BD78680007800F55
:100D5000F3D115480168C907C90FB1420BD9016821
:100D600049084900314301600068C007C00FB04224
:100D700001D00120F8BD2078400706D5786807210A
:100D800009028843E1680843786000F01DF879683B
:100D9000084A0906090F515CC8400749086000204D
:100DA000FFF7C8FE0020F8BD0020024000100240FE
:100DB0008813000005530008FC000020014800686B
:100DC00070470000FC00002010B513A00FC888B0C9
:100DD0006C460FC414A00FC80FC4174B5A680C20E0
:100DE00011460140154804290FD008290DD1910260
:100DF000090F6C46645CD96A04AB0907090F595C9A
:100E0000D20304D5FFF770F9604308B010BD0C4958
:100E100020464843F9E700000203040506070809D5
:100E20000A0B0C0D0E0F1010010203040506070833
:100E3000090A0B0C0D0E0F100010024000127A0070
:100E400000093D00042204490428086902D09043A7
:100E5000086170471043FBE700E000E00F480168BD
:100E6000643101600E480168491C01600D49086841
:100E7000401C08600C490D4A8868401C88609042FC
:100E80000BDB002088600A48816F491C8167016F75
:100E9000491C0167416F491C4167704724000020CD
:100EA0001C00002074000020D0000020102700004B
:100EB00098120020094910B5401E884201D901202E
:100EC00010BD074C60610321081F02F0C9F8002023
:100ED000A06107202061002010BD0000FFFFFF007F
:100EE00000E000E010B5FFF7B9FF10BDFEE700001D
:100EF000002110B5104A012308469B0251601418C6
:100F0000401C21729842FADB002009230B4A9B0106
:100F10004400A418E418401CA1861028F8DB002027
:100F200011239B014400A418E418401CA182FF284F
:100F3000F8DD002010BD000024170020980A0020D2
:100F4000402802DB0020C043704710221143C2003A
:100F5000094B4000D218C0180D2311879B010021B6
:100F6000C31899820B239B01C01881820348006833
:100F70005063084670470000980A002000010020D6
:100F800070B504461E464430049D03F029FD2046FA
:100F90002A463146643003F023FD002070BD000076
:100FA00070B5104D064601462846FFF7B3F80E4CC3
:100FB0002061FFF703FF2946FFF796F8A0600B4872
:100FC000314600680546FFF78FF8E0602A460023A7
:100FD00007480F21FFF7B2F8208020696430606075
:100FE000002070BD40420F0020000020FC000020C7
:100FF00000004042704700B502F000FC00BD7047A1
:10100000332E303000000000FEB504460078D04D8D
:10101000C00746D068680007800F012807D06868BD
:101020000007800F022809D16868C00306D5286828
:10103000800336D5606800287ED032E001216068E8
:10104000090401280AD08A00002801D005280FD001
:101050002868884328602868904301E0286808438E
:1010600028606068002810D0FFF746FD064608E0BB
:10107000286810432860F1E7FFF73EFD801B6428D5
:101080006FD828688003F7D50BE0FFF735FD0646DB
:1010900004E0FFF731FD801B6428F1D82868800345
:1010A000F7D420780126800700283BDA686800071B
:1010B000800F07D068680007800F022809D1686890
:1010C000C00306D42868800715D5E068012833D10D
:1010D00011E0E0680028286815D030432860FFF749
:1010E0000BFD074604E0FFF707FDC01B0228C7D829
:1010F00028688007F7D52868F82188432169C90046
:10110000084328600EE0400840002860FFF7F4FC28
:10111000074604E0FFF7F0FCC01B0228B0D828689F
:101120008007F7D42078000724D5E0690028686A92
:1011300010D03043686200E007E1FFF7DDFC0746AE
:1011400004E0FFF7D9FCC01B022899D8686A800721
:10115000F7D50FE0400840006862FFF7CDFC074676
:1011600005E09DE0FFF7C8FCC01B022888D8686A2C
:101170008007F7D4207804274007002860DA002091
:101180000190E869C00008D4E969B8060143E96143
:10119000E96901400120009101906E480168C9058C
:1011A00011D40168821511430160FFF7A5FC00907E
:1011B00005E0FFF7A1FC0099401A642870D8654843
:1011C0000068C005F5D5A06801280AD0002801D024
:1011D000052810D0286A400840002862286AB843D1
:1011E00001E0286A30432862A068002812D0FFF787
:1011F00083FC00900AE0286A38432862F1E7FFF791
:101200007BFC0099411A5448814249D8286A8007DA
:10121000F5D50DE0FFF770FC009006E0FFF76CFCE1
:101220000099411A4C4881423AD8286A8007F5D47F
:101230000198002804D0E969012000078143E96191
:101240002078C00635D5606901280CD0401D686B38
:1012500023D038436863686B400840006863FFF739
:101260004BFC064622E0686B38436863686B30438A
:101270006863FFF741FC064604E0FFF73DFC801B76
:1012800002285BD8686B8007F7D5686BF821884324
:10129000A169C900084368630BE0B8436863F4E7D9
:1012A0004CE0FFF729FC801B022847D8686B8007B9
:1012B000F7D4206A002846D069680907890F0229F7
:1012C00043D001273F060228286805D0B84328608C
:1012D000FFF712FC044633E0B8432860FFF70CFC2C
:1012E000064604E0FFF708FC801B022826D8286881
:1012F0008001F7D4E86AE16A000900010843E86266
:10130000616AA06A084369683D2212049143084358
:101310006860286838432860FFF7EEFB044604E065
:10132000FFF7EAFB001B022808D828688001F7D5E0
:1013300009E0FFF7E1FB001B022801D90320FEBDF5
:1013400028688001F5D40020FEBD0120FEBD00000C
:1013500000100240007000408813000030B50022E9
:1013600072B610210925ED06A962A961431E01216B
:101370009940084C002809D023681B0600D40A4372
:101380002023AB624908AB61401EF5D162B610461E
:1013900030BD000010000048F8B572B610210925D4
:1013A000ED06A962A961C117490F0818C7100020EE
:1013B0000C4E034600900FE0002280210820346884
:1013C000640600D40A432024AC624908AC61401E84
:1013D000F5D16846C2545B1CBB42EDDB62B6009897
:1013E000F8BD000010000048034610B5002002467A
:1013F00002E09C5C6040521C8A42FADB10BD000097
:10140000F0B5224F6024F8780E466043204C0B78EC
:1014100000210019C9431F4C252B06D06269521CBC
:101420006261C269521CC26108E07579802D07DDD6
:10143000A269521CA261026A521C02620846F0BDF7
:10144000294608318A4208D2016A491C0162A06912
:10145000401CA0610220C043F0BD3046A91DFFF72B
:10146000C3FF7119897981420DD0E069401CE061A8
:10147000F9786020414306480818416A491C4162D6
:101480000320C043F0BD0020F0BD00005800002044
:101490006405002024030020F8B50E4604462520EC
:1014A000069F079D089920706270A670E3702771EF
:1014B0002F46002008376619372B1AD009DC1A4648
:1014C000303A130002F09EFF072615152626261730
:1014D0002600612B0DD006DC382B0AD0412B08D01A
:1014E000422B17D105E0622B03D0632B01D0642B74
:1014F00010D1657102E06571002D03D02A46A01D50
:10150000FEF753FEA91D2046FFF76EFFB0710D20B8
:10151000F0713846F8BD0000F1B584B0FFF7ECFA81
:101520000546FFF71BFA544E04467079002806D092
:10153000B079002803D0F068201A322805D8F06866
:101540007D21201AC90088427ED9B0794B490028F4
:101550001DD0F27860235A43494B012098506420F3
:101560004866F078401CC0B2F070717A884208D9A1
:10157000B06AB462201AF0623079401C30710120E8
:10158000F0704048008A404F002828D031E0706A4F
:10159000401C70623D480269521C0261F378602071
:1015A0009C464343364818180269521C026142693E
:1015B000521C42617779002F02D1876A7F1C8762B3
:1015C0008769BA4200D982612D48032AC9D900220D
:1015D000C250C82088662E4960460A54C1E7FFF70A
:1015E00045F9294980B240398886C1B2F982000A9A
:1015F00038832749B87D10314870387E8870F2787A
:1016000024488B5C037089184978417060211C4B19
:101610005143595C81700027C7700571290A4171D7
:10162000290C8171290EC171F4603379029008216F
:10163000174800930191412339462030FFF72CFFD2
:1016400013490246203100E012E0049802F03EFA0D
:10165000F078602148430A4940184168491C4160BC
:10166000C268F1688A1A4263C16075637771B771A5
:10167000002005B0F0BD00005800002098120020A6
:1016800064050020EC140020D80C00202403002066
:101690004404002064080020F7B54E4D4A7986B016
:1016A0000C46E8786021049048434B49A31D40183C
:1016B0008168491C8160484980390391A178E678A6
:1016C00001932B461F6BDB68303EFF1A2B469B694C
:1016D0000093330002F096FE13420B174242422958
:1016E000424242424242424242422C4542003B4830
:1016F000A3794354217901983223019200910290F9
:101700000021049A22E06F61009A974200DDAF61E8
:10171000324AA37953540021C7624161016BB94237
:1017200000D207630120A87118E00120687115E05C
:101730002A48A179017010300078A07121790198B0
:101740000192009102904223A97800220398FFF7AA
:10175000A3FE02460399069802F0B8F9002009B0EA
:10176000F0BD6F610098874200DDAF611B4AA07930
:1017700050544A001A495118FF31FF31023188860E
:101780001848008A00280AD11748C18E008F00022D
:101790000818154980B240318882FFF72CFCEA789E
:1017A000602042430C480021161871616869F0629C
:1017B000316B814200D230632046677A0A30FEF7EF
:1017C00018FD617B0002000A09060843B900711880
:1017D0008863A7E758000020640500204404002027
:1017E000980A0020EC140020980C0020F7B516464B
:1017F0000F46FFF7B3F8164C20632178002000292C
:101800000FD001256571324639460098FFF7F8FD83
:10181000002805D1A571324639460098FFF73CFFF4
:10182000FEBD61780029FBD00A4C3246A06B3946D8
:10183000401CA063009800F011F80028F0D1064881
:101840003246406E20653946009800F073F8FEBDC0
:10185000580000206405002098120020F0B50E46C4
:10186000087800211A4FC9431A4C252806D0606910
:10187000401C6061386C401C386409E0144875797C
:10188000806C401C802D05DDA269521CA261B864E9
:101890000846F0BD294608318A4206D2B864A069DC
:1018A000401CA0610220C043F0BD3046A91DFFF7D7
:1018B0009BFD71198979814208D0E069401CE06183
:1018C000F86C401CF8640320C043F0BD0020F0BD5C
:1018D0006405002024030020F8B5FFF73FF8124B01
:1018E0001A69DC791149002C05D07D2080014866F9
:1018F0000020D87115E00D4E0D4C851A8036A5429A
:1019000004D97D2292018A66012106E012199042D3
:1019100007D97D2292018A660221B161F0611869BE
:1019200030620020F8BD000058000020981200200E
:10193000E02E0000F7B557480C46C16884B0491C3A
:10194000C160657960785449544A03919178277948
:1019500088420AD0FF2808D04F488030416C491C8B
:1019600041640020C04307B0F0BD884201D0FF2889
:101970007ED1106B009010610120D071E078A61D1F
:10198000372875D007DC3038030002F03BFD0681B4
:1019900013818181228161287AD004DC382877D0B4
:1019A000412875D126E0622872D0632870D064285F
:1019B0006ED162E03848A379A03803701030007807
:1019C000A0710098106120796F4661C73223002210
:1019D00006E0002036230190024601210097029084
:1019E0000398FFF759FD02462B488030C16B491C14
:1019F000C1633BE02849A079A0390870E37AA17A55
:101A00001B02CB182549CB61FFF7F5FA2348077A6B
:101A1000FEF72CFF204990390870A0716772B8005A
:101A20001D4F8037C019018FA172018F090AE17221
:101A3000816B090C2173806B1849000E6073174885
:101A4000007A401CC0B208720A2801D30020087234
:101A50002079694661C111484223817800220398A8
:101A6000FFF71AFD0246F86B401CF863039900E08B
:101A70000EE0049802F02AF80AE0E179A079090260
:101A80004018217A637A09041B06C9184018D061EE
:101A9000002068E724030020E40400205800002010
:101AA000034610B50020024602E09C5C6040521CD8
:101AB0008A42FADB10BD30B50D4608460978144657
:101AC000252901D0012030BD062C01D2032030BDD4
:101AD000611EFFF7E5FF29192039C97F814201D036
:101AE000042030BD002030BDF8B51E460B465527FA
:101AF000069D0799077043708270C6700446057191
:101B00002A46401DFEF751FB691D2046FFF7C8FF1E
:101B1000014660194171A81D052E02DA002E00D180
:101B20000020F8BDFEB516460F460546FFF7C3FF79
:101B3000040014D0684604720420009002A90B48E7
:101B400001910278401E0178EE230948FFF7CCFF8F
:101B500002460749284601F0B9FF2046FEBD32463D
:101B60003946284600F006F8FEBD0000950000202A
:101B7000F4080020F7B5FC480C464D7886B0416863
:101B80008160411C0A78A678120936071201360FC7
:101B9000237932430A70F549029100780490854216
:101BA00001D0FF2D28D1E078F14E312865D024DC1A
:101BB000F04F172839687DD010DC05285DD006DC91
:101BC000002819D0012835D0032874D138E007281F
:101BD00020D01128F5D01628F7D1E4E122286BD0C7
:101BE00006DC182869D0192868D02128EDD115E124
:101BF0002328E6D02428E8D169E20421632872D0A2
:101C00000EDC552870D006DC322803D0332834D0BF
:101C10003428DAD194E0562867D05728D5D11DE270
:101C20000646643E330002F0EDFB08F0EF161A465C
:101C30000E461446641D00932946019401233EE29A
:101C4000CD4B102124E2CD4B0C2121E22946034645
:101C500035E2CB4B1CE2CA4B103B502118E2E17934
:101C60000020C24A03E023185B7A1354401C8842C8
:101C7000F9DBBE4802F034FB89E0A77961793F02C5
:101C8000C919E479882B21D0892B23D08A2B25D020
:101C9000832B2BD0842B2ED0852B31D0862B34D088
:101CA000872B37D08B2B3AD08C2B3DD0FE2B11D0ED
:101CB000992B04E08EE10DE2FCE095E1B4E138D02F
:101CC000A12B39D0A94B103B59187DE149008B1944
:101CD000AC49F9E749008B19AB49F5E749008B1985
:101CE000A8492039F0E7D2E1BBE1C5E149008B19F1
:101CF0008D218900E8E749008B1995218900E3E7E8
:101D000049008B199D218900DEE749008B19F521D7
:101D10008900D9E749008B19FD218900D4E74900E2
:101D20008B19D5218900CFE749008B19B52189008E
:101D3000CAE74B009549C7E74B000121C906C3E735
:101D4000A179607909024018E279882B28D0892B83
:101D50002AD08A2B2CD0832B2FD0842B32D0852BCA
:101D600035D0862B38D0872B3BD08B2B3ED08C2B7D
:101D700041D0FE2B44D0992B48D0A12B49D07B4990
:101D800010390818002221460931FEF70EFA00200A
:101D9000009001907448E378401C027829468EE157
:101DA00040008119774837E040008119764833E0D8
:101DB00040008119734820382EE0400081198D20A1
:101DC000800029E0400081199520800024E0400037
:101DD00081199D2080001FE040008119F5208000BE
:101DE0001AE040008119FD20800015E040008119B3
:101DF000D5208000C5E740008119B5208000C0E7EC
:101E0000400081196048BCE750E144E141005F486F
:101E100002E041000120C0060818B4E7A17960790A
:101E200009024018002B12D009218901012B19D079
:101E3000022B25D00F218901032B13D0042B1FD097
:101E4000052B22D0062B20D0082B2CD008E0011126
:101E500049008919FF31FF31023109E0012019E001
:101E6000002017E003115B009B195918898A00E0D4
:101E7000898E03071B0F012098400142F0D0EDE747
:101E800003115B009B195918F2E7C0008019008FFD
:101E90004006C00F6946087303A901200191009014
:101EA000294621230BE101114900012389199B02D5
:101EB000C918DDE7A179607909024018002B1BD011
:101EC000012B22D0022B29D0032B30D0042B37D06A
:101ED0004021052B3DD0062B3BD0072B58D00020AE
:101EE00069460873002000901F4803A90191401C17
:101EF000027829462223E2E00107001140008319FD
:101F0000090F8D20E279800049E0010700114000AF
:101F10008319090F9520E279800040E00107001144
:101F200040008319090F9D20E279800037E0010706
:101F3000001140008319090FF520E27980002EE09E
:101F40000107001140008319090FFD20E27980008C
:101F500025E0C0008019028F8A43E179C907490E44
:101F60000A430287BEE7000094000020F408002026
:101F7000980A0020241700201C520008ACF7FF1F0D
:101F8000107C00085404000054080000F4090020EC
:101F900001070011090F40008319E279524818180F
:101FA00001F0BAFD9EE7A679617936028919E479D4
:101FB0004E4E002B0BD04E4F012B03D04D4B9B8A26
:101FC000002B04D04900C919009401913EE6490054
:101FD0008919F9E7002901D000203860002000901D
:101FE0002946172301906AE0002901D000203860BB
:101FF000A179607909024618E27900203E4903E0A0
:1020000027187F7A0F54401C9042F9DB3A4930463A
:1020100002F070F9002009340090019037480394D1
:102020000278294618234AE0A1796079090241180B
:102030003048C182818A00290ED0002181822D483A
:1020400001F004FD012038600020009001902B4831
:1020500029460278192332E00121EFE7254B2021A0
:1020600016E0274802F066F900200090019023480E
:1020700029460278552322E01E4801F0E7FC0020A3
:10208000009001901D4829460278562317E01D4B09
:1020900001930091DAE5A179607909024018E179AC
:1020A0000E01FEF7D1FBF1B2009172E6FEF7E6F900
:1020B000002000900190114829460278652302987B
:1020C000FFF712FD02460299069801F0FFFC00207E
:1020D00009B0F0BD02206946087303A901200191EF
:1020E000EE2300900499EAE7340400000080000821
:1020F00000A00008EC140020F40800209500002047
:10210000F40900202C13002070B5FEF781F9164861
:1021100000F096FA154D164E6869B067124881684E
:1021200071678188491C81808088F0660E4801F0C3
:102130008DFC344680342868206168686061A86836
:10214000A06101220B4B1146B06FFEF705F9E8685C
:102150002062A8696062E869A0622869E062286A72
:102160002063002070BD0000EC140020A0000020BF
:10217000981200203930000030B5836801221340E6
:1021800002D00022104630BD8C684B68C9682343DA
:10219000C468034D2C4021430B43C360F2E70000A9
:1021A000C73FFFFF30B583680122134002D00022F1
:1021B000104630BD18C94D6823430C6889682C430C
:1021C00023430B43C168024C21400B43C360EFE73C
:1021D0003CC2FEFF08B504494A6902434A614969A5
:1021E0000140009108BD00000010024008B50449FC
:1021F000CA690243CA61C9690140009108BD000073
:102200000010024008B504498A6902438A6189695D
:102210000140009108BD00000010024070B5094E59
:1022200004467618203E049D0C34F17F0830102DB2
:1022300003D00A50F07F035170BD0A51F17F0B505B
:1022400070BD0000164E0008044A51182039C97F9D
:10225000425852085200425070470000164E000883
:10226000044A51182039C97F425801231A43425069
:1022700070470000164E0008044A51182039C97FE3
:10228000425802231A43425070470000164E00087D
:10229000054B10B559182039C97F4358032424032E
:1022A000A3431343435010BD004E0008054B59187B
:1022B0002039C97F001D0B581B0C1B0413430B5006
:1022C00070470000164E0008054B10B5591820390C
:1022D000C97F4358034C23401343435010BD0000B3
:1022E000004E0008EFBFFFFF054B10B5591820390D
:1022F000C97F43588024A3431343435010BD0000BB
:10230000004E0008054B10B559182039C97F4358B5
:102310000324A402A3431343435010BD004E0008FE
:10232000054B10B559182039C97F43582024A343C1
:102330001343435010BD0000004E0008054B10B57C
:1023400059182039C97F43584024A34313434350AD
:1023500010BD0000004E0008054B10B5591820397B
:10236000C97F435803242402A3431343435010BDA1
:10237000004E0008F0B500233CE001249C402240C0
:1023800037D04F6806681446544365006519AE435C
:1023900067433E4306604E68012E01D0022E05D1F0
:1023A0008F6886686743AE433E4386600F69C668A0
:1023B000AE4325467D432E43C6604D68022D18D19D
:1023C0004D69FF2A09D8066A544354432201121B5F
:1023D00096436C43264306620BE0140A224662438E
:1023E000624362431401A61A446A6A43B443144325
:1023F00044625B1C0A681446DC40BED14A68012A6C
:1024000001D0022A06D10A68C968436893434A4347
:10241000134343600120F0BD10B5044601F05AFAA1
:10242000206001F03DFA606001F048FAA06010BD44
:10243000014610B5002000290FD1104A116B890701
:10244000890F01290AD0022911D0032909D001F0EE
:1024500041FA01F025FA01F031FA10BD01F03AFA23
:1024600010BD11688907C90FFAD0054810BD116A5F
:102470008907C90FFAD00120C00310BD0010024027
:1024800000127A0010B5036800225B06DB0F25D12D
:102490000CC98C681A434B6823431A43CB681A4310
:1024A0000B691A434B691A438B691A4303680C4C36
:1024B00023401A43026042680A4B1A40CB681B0C47
:1024C0001A430B681A43426001238A695B03083987
:1024D0009A4202D1898C89B201610122104610BD55
:1024E0004000FFFFFBF0FFFFF0B50268194B1A4CEC
:1024F000984201D0A04203D17025AA434D682A43D7
:10250000164D174E174F98420AD0A04208D0164CCD
:10251000A04205D0A84203D0B04201D0B84204D1B5
:1025200003242402A243CC68224302608A68C26268
:102530000A888262984205D0A84203D0B04201D0F6
:10254000B84201D1097C0163416901221143416113
:102550001046F0BD002C0140000400400040014046
:102560000044014000480140002000404168012231
:10257000D202914341608168082291438160704793
:10258000FEB5044600680D460026C007C00F43D1C3
:10259000E9686868AA690843296911430843216802
:1025A0001E4A114008432060A86861680322120394
:1025B0009143014361606869A1681211914301432D
:1025C000A1601748844203D10020FFF731FF06E0E5
:1025D0001448844220D16846FFF71EFF0298002865
:1025E0001AD02968002917D00126AA69F3039A4254
:1025F0000CD140004A088018FDF776FD0A4980B2E8
:1026000001400007420F0A43E26005E04A08101843
:10261000FDF76AFD80B2E0603046FEBDF369FFFF62
:102620000038014000440040F0FF000010B59C223B
:102630000249FDF7BAFD002010BD00002C52000831
:10264000F0B5134A00215514124C134F0CE0D65A22
:10265000BE4208D19B185B886668B34203D90AC49E
:102660004B1C2360083C491C4B01AB42EFD3216853
:10267000002904DB49018918202201F061F9A068D2
:1026800040012030A84201D90020A0600020F0BD08
:1026900000A80008A0000020AA5500001FB50B46A6
:1026A000024604A1684601F099FE0146684601F021
:1026B000D5F81FBD201B5B25643B25644800000046
:1026C00070B501208AB04002FFF79CFD224CA06A41
:1026D00003263043A0622149B0050A6882430243C1
:1026E0000A60A26A83111A43A2620A688243024303
:1026F0000A60002505950695079505A920460895C9
:10270000FFF73AFD01200390009501950295694677
:1027100004952046FFF746FDE16804208143E1600F
:102720006169C908C9003143616161680143616041
:102730006068082188436060A06817218843C90742
:102740000843A060A068C00FFCD1A06804490840FD
:10275000401CA0600AB070BD002401400827014061
:10276000E8FFFF7F10B50120FFF734FD00210A20AC
:1027700000F054FC0A2000F047FC00210B2000F080
:102780004DFC0B2000F040FC10BD0000F0B5012016
:1027900087B04004FFF71EFD01208004FFF71AFDFB
:1027A0000120C004FFF716FD01208005FFF712FD90
:1027B0000126C020002403256A46049631C2092759
:1027C000FF0669463846FFF7D5FD8020694631C1CE
:1027D000694638460494FFF7CDFD93200001009030
:1027E000039469460196029504943846FFF7C2FDAA
:1027F0003002B86168026A46049631C269463846BA
:10280000FFF7B8FD0F486A46049631C20E4F69467D
:102810003846FFF7AFFD0D480090039469460196D6
:10282000029504943846FFF7A5FD07204003009069
:10283000029403946946019604940548FFF79AFDB3
:1028400007B0F0BD0704000000040048EEBC000023
:102850000008004808480749016008490160042150
:102860004160074A8260C1684907FCD1026105499D
:1028700001607047CCCC000000300040555500008E
:10288000FF0F0000AAAA0000F0B591B0282106A809
:10289000FDF7A4FC18216846FDF7A0FC01263603CD
:1028A0003046FFF7AFFCB001FFF794FC002408208E
:1028B00002250327039404946A460594A1C269463D
:1028C0001F48FFF757FD102069460394A1C101205E
:1028D0000490694605941A48FFF74CFD20200394A4
:1028E00004946A460594A1C269461548FFF742FD63
:1028F0000021192000F092FBFF20053007900720EF
:1029000000020890069428020B90099408200A946B
:102910000D940E940C9007200A4C0F9006A92046A7
:10292000FFF7B0FD60681021884360606068B043C5
:1029300030436060206840210843206011B0F0BD42
:102940000004004800300140F0B591B0282106A8ED
:10295000FDF744FC18216846FDF740FC0127BF0342
:102960003846FFF743FC3801FFF734FC00247810A9
:1029700002250326039404946A46059461C26946BD
:102980001C48FFF7F7FC0097039404946946194824
:10299000029601950594FFF7EDFCA80303940494B7
:1029A0006A46059461C269461248FFF7E3FCFF20BE
:1029B0000530079007200002089006940994280229
:1029C0000A940C940D940E940B9007200A4C0F90CF
:1029D00006A92046FFF756FD606810218843606015
:1029E0006068082108436060206840210843206037
:1029F00011B0F0BD000400480038004010B586B0AA
:102A000014216846FDF7EAFB1020FFF7EFFB0021D9
:102A1000112000F003FB112000F0F6FA2F20694688
:102A20000880002001900848084C02902046FFF7DB
:102A30005BFD2068802188432060E0680121084315
:102A4000E06006B010BD0000E70300000010004089
:102A500070B501208EB08003FFF7D4FB0320400245
:102A600007900220089003200024099001250920E6
:102A70000A9407A90C950B94C006FFF77BFC3A4E0D
:102A8000102202213046FFF71FFC002202213046AF
:102A9000FFF7FEFB002202213046FFF741FC002237
:102AA00002213046FFF74AFC802202213046FFF720
:102AB0001BFC002202213046FFF74EFC00220221BF
:102AC0003046FFF71FFC002203213046FFF7FCFBD6
:102AD000002203213046FFF7DBFB002203213046B2
:102AE000FFF71EFC002203213046FFF727FC80225F
:102AF00003213046FFF7F8FB002203213046FFF7A1
:102B00002BFC002203213046FFF7FCFB00211B2099
:102B100000F084FA1B2000F077FA14486946006838
:102B20000090019402940394059406940C20104C98
:102B300004902046FFF724FD606829050843606083
:102B40006068490003225205904308436060A06812
:102B500049120843A0602046FFF708FD206828437B
:102B600020600EB070BD0000000002403800002060
:102B70000038014070B58EB01C216846FDF72EFB71
:102B8000182107A8FDF72AFB012464042046FFF75B
:102B90002DFB2046FFF71EFB0E2007900220089019
:102BA000032000240990012609200A9407A90C9605
:102BB0000B94C006FFF7DEFB414D1022042128468E
:102BC000FFF782FB002204212846FFF761FB002269
:102BD00004212846FFF7A4FB002204212846FFF722
:102BE000ADFB802204212846FFF77EFB0022042152
:102BF0002846FFF7B1FB002204212846FFF782FB9D
:102C0000002205212846FFF75FFB00220521284608
:102C1000FFF73EFB002205212846FFF781FB00223B
:102C200005212846FFF78AFB802205212846FFF769
:102C30005BFB002205212846FFF78EFB00220521C1
:102C40002846FFF75FFB00211C2000F0E7F91C205D
:102C500000F0DAF9A51EFF21284600F0DFF928462A
:102C600000F0D2F91748F50300680090019402942F
:102C700003940C2004AA31C2134C69462046FFF786
:102C80007FFCA06821140843A060A068A8432843E3
:102C9000A06020681F214905884308432060206800
:102CA0004911884308432060A068A1140843A0602C
:102CB0002046FFF75BFC2068304320600EB070BDFB
:102CC000000002403C0000200044004000B50846DF
:102CD000042A02D80020C04300BD01787F2902D910
:102CE0000120C04300BD41784906490E1F2902D981
:102CF0000220C04300BD114601F022FE0028F9D099
:102D0000042000BDF7B588B00F460A9A0898FFF76F
:102D1000DDFF0690002803D00020C0430BB0F0BDBB
:102D2000B6483A780078394682427DD18C784A7824
:102D3000CB78B98824024DBAB1491C4308704A7057
:102D400001200790200521070226000E090F13001D
:102D500001F058FB119E0A47859FB7D59E9E9E9E07
:102D60009E9E9E9EE1F39E00E81DC008A44903902C
:102D7000887000202FE00020009001200190029830
:102D80000027C00004901CE02005000E42009D4872
:102D900021071218092080011018090F808AFDF7F9
:102DA000D1FC002803D001990098084300900198B5
:102DB000641C4006000E7F1CA4B20190082F03DAA9
:102DC0000498C019A842DFDB8D49029A009889183F
:102DD000C8700298401C039902908842CBDB761899
:102DE00055E0E81DC008864903908870002031E056
:102DF000002000900120019002980027C00004905C
:102E00001EE02005000E42007E4821071018FF300A
:102E1000FF300230090F808EFDF794FC002805D0AA
:102E200001990098084300E0E5E000900198641CD7
:102E30004006000E7F1CA4B20190082F03DA04980C
:102E4000C019A842DDDB6E49029A00988918C87043
:102E50000298401C039902908842C9DBBFE76800D2
:102E600067498446887000200EE021184A006549B1
:102E700047005218112189015118898A604A0B0AAA
:102E8000BA18D3701171401CA842EEDB17E0761C13
:102E900087E068005A4A8446907000200DE02118AF
:102EA0004B00584947005918FF31FF310231898ED4
:102EB000BF180B0AFB703971401CA842EFDB664457
:102EC000E5E7002D12D0FF221202954207D1420001
:102ED0004C48121895208000101800F015FE394655
:102EE00047480A9AFDF761F90A9E7FE0420045488B
:102EF000121895208000101800F06EFDEFE7387969
:102F00007979000208433F49620052181121890172
:102F100051188882E3E7E81DC0083949039088709A
:102F2000002030E03818C079009001200190002086
:102F300005900298C00004901FE036E02005000EC6
:102F400042003048210712189520090F8000101800
:102F5000009B019A1A4202D000F0D6FD01E000F079
:102F60003BFD0198641C4006000E01900598A4B238
:102F7000401C0590082804DA049805994018A842D6
:102F8000DCDB0298401C039902908842CADB1C4893
:102F9000B9788170F978C1703979017179794171A5
:102FA000361D0698002814D025E000200EE04100D0
:102FB000C919CA79097A12020A4321184B0011492A
:102FC0005B181121890159188A82401CA842EEDB46
:102FD000DDE70798002809D0B1B2094801F0B0FC3C
:102FE00007498855000A89194870B61C32460449B9
:102FF000089800F06BFD002090E60000F40000202F
:10300000A4160020980A0020C106C90E012088409D
:10301000014908607047000000E100E08307FF22DB
:10302000DB0E9A408907090E994000280BDA000749
:10303000000F0838830808489B001818C369934399
:103040000B43C3617047830804489B00181803684A
:1030500093430B430360704700ED00E000E400E0A1
:103060008307FF22DB0E9A408907090E994000284A
:103070000BDA0007000F0838830808489B0018186F
:10308000C36993430B43C3617047830804489B00A3
:103090001818036893430B430360704700ED00E08A
:1030A00000E400E010B501200449C006486004486F
:1030B0000168491C016000F005F810BD00ED00E05A
:1030C0003400002070B5094CA06800280CD0084DD1
:1030D000084902202A68FEF789FB00202860A060CA
:1030E0008021044801F072F870BD00002403002024
:1030F00044000020C403002010B50648054B0078AA
:103100000021203B5A1820325478491C14700F2992
:10311000F8DB10BDB80A002010B5094C094B01229C
:103120000221A06FFDF718F9074800F08FFCE06F4F
:103130002146401CE0678031A06F0860002010BD70
:103140009812002039300000EC1400200248C16FB2
:10315000491CC1670020704798120020F3B5F84D54
:1031600085B0286800286FD0686800281CD000222D
:103170000D21082000F0E8FC00221146082000F094
:10318000E3FC01221146082000F0DEFC002001468D
:10319000EC4A13182033401C19701028F8DB002665
:1031A00001211446203467E20122E1E7B2000598CC
:1031B000059B805CD7187A78019201257B88009363
:1031C0001B2873D012DC0246030001F01BF91B5CC4
:1031D0007272727272723E3E3E3E3E3E5C5C5CA714
:1031E000A7A73E3EBEBEBEBEBEBE5C00342870D0A9
:1031F00011DC01461C390B0001F004F918A7A7A740
:10320000A7A7A7A7A7A7A7A745454545454545455E
:1032100045454545F7453A2873D008DC0146353920
:103220000B0001F0EFF805E26E56E26E3000DC288C
:1032300004D004DC3B28EFD0C82824D120E1DD28CD
:10324000FCD0FA28F9D11BE11FE2D01F030001F0E6
:10325000D9F80E080A10181B1D1A1A1A1A1A1A2061
:10326000261A207C4AE0FFF747FF00281FD0207C69
:103270003AE0FFF741FF002816D1207C002813D147
:1032800025E000F0ABFAF1E12078F7E7FFF734FF33
:103290001DE0207C00280AD0002905D007E0207C12
:1032A000002804D1002902D0012010E04DE00020C8
:1032B0000DE0130001F0A6F8070C050E111B262ED9
:1032C0000C0000F08BFA00990198FDF745FA207484
:1032D000CCE116E100F082FA0CE0207C0028E6D078
:1032E00000990198FDF738FA0028E0D0DCE7207C4F
:1032F0000028DCD000990198FDF72EFA0028D6D1DD
:10330000D2E754E1207C0028CED100990198FDF746
:1033100023FAB3E7207C0028ECD0C5E7102804D0BE
:10332000112804D0122AAED10AE0227C03E0207CCE
:103330000028A8D001220099019800F005FC95E131
:10334000207C00289FD00022F5E715383D79030046
:1033500001F058F8120A1215181B0F1E3C4C5B6A3C
:103360002D798185898D7D9400F038FA13E02074E1
:1033700084E000F033FA1DE000F030FA29E000F0BC
:103380002DFA36E000F02AFA42E000F027FA4EE08B
:10339000207C002870D028460099FDF76DFA05467C
:1033A000F9887879FDF768FA854263D064E0207C7B
:1033B000002861D028460099FDF75EFA0546F98895
:1033C0007879FDF759FA854254D155E0207C0028E0
:1033D00052D028460099FDF74FFA0546F9887879CA
:1033E000FDF74AFA854245DB46E0ADE0207C002847
:1033F00042D028460099FDF73FFA0546F9887879CA
:10340000FDF73AFA854235DC36E0207C002833D0DF
:1034100028460099FDF730FA0546F9887879FDF7D6
:103420002BFA854226DD27E0207C002824D0284680
:103430000099FDF721FA0546F9887879FDF71CFA1D
:10344000854217DA18E0207C002813D1A3E7207CFE
:1034500000280FD1AEE7207C00280BD1B9E7207CF3
:10346000002807D1C5E7207C002803D1D0E7207CC5
:103470000028DCD001207AE7002078E70225F5E07B
:103480003F791546C8280CD0DC2821D0DD2827D06C
:10349000FA28F3D12B48E9000818008FC00627D579
:1034A00007E02848E9000818008FC00601D4002171
:1034B0001FE0207C002820D038460099FDF7DCF979
:1034C0000146284600F090FA284600F0E3F84EE75F
:1034D0001C48E9000818008FC006EAD4012108E062
:1034E0001848E9000818008FC006E2D4022100E065
:1034F00003212846FDF724FDDBE7284600F0E8FC21
:10350000E2E73F790225342802D0372816D108E0B7
:10351000207C002812D038460099FDF7ADF9401CF8
:1035200007E0207C002809D038460099FDF7A4F96F
:10353000401E02463846009900F070FB96E00000FD
:1035400024170020980A00203D7979790291F988A2
:103550000191332814D035281BD038288ED1207CF7
:1035600000288BD00298FDF787F907462846009976
:10357000FDF782F93A1A0199029800F04FFB7DE7B6
:10358000207C0028FBD028460099FDF775F90246FB
:10359000F1E7207C0028F2D028460099FDF76CF96D
:1035A000054601990298FDF767F92A18E3E73A7989
:1035B00079790291F9880191797A03917D89362888
:1035C00006D0392812D03A281FD03B284DD131E0FF
:1035D000207C002849D010460099FDF74DF9074698
:1035E00001990298FDF748F93A180CE0207C002870
:1035F0003BD010460099FDF73FF907460199029824
:10360000FDF73AF93A1A29462CE0207C00282CD004
:1036100010460099FDF730F907B201990298FDF7BD
:103620002BF900B247433A462946039800F0F6FAD0
:103630003A1416E0207C002817D010460099FDF7B8
:103640001BF907B201990298FDF716F901B2384645
:10365000FCF760FD02B20F462946039800F0DEFA3F
:103660003A46691C039800F0D9FA03250848227CE1
:103670008019017A027276190698864200DA95E579
:1036800003494868401C4860002007B0F0BD0000B6
:1036900024170020F8B50746402802DB0020C0436D
:1036A000F8BD2A48F9000D182C8FE10601D400203E
:1036B000F8BDA1063AD561063DD425490968686B75
:1036C0000090081A0A26A1070FD0A107890F012927
:1036D00005D0022905D0E143890705D005E064261D
:1036E00003E07D26F60000E01A4EB04223DB3146AF
:1036F000FCF710FD014615487A0012180B208001D6
:1037000010188446808A009B4018714359186963D9
:103710000D2189015118898A80B2814203D8084657
:1037200040210C432C876146888204E0600602D564
:10373000402084432C87288FB9B24006C20F052051
:1037400000F002FA288F4006C00FF8BD980A00204A
:103750000001002010270000F7B50446FDF761F8CE
:10376000054602992068A942A16806DC4018029A21
:103770000199FCF71AFD029919E040182A460199AF
:10378000FCF713FD29462046FCF72CFE2046FDF7EA
:1037900048F806460298471BB7420DDCA16820682E
:1037A0003A46401801994919FCF7FFFC3946204672
:1037B000FCF718FE0298FEBD002E0CDDA168206803
:1037C0003246401801994919FCF7EFFC3146204672
:1037D000FCF708FEAD192846FEBD0000064A0F2082
:1037E0001118CB7F2031401E0B700028F8DC0249F5
:1037F0002031087C08707047980A002070B572B6B6
:103800000124134D2403AC61124A010A11730026EE
:1038100091688907C90FFBD00F4B00215E6400E05F
:10382000491C96683606F60FFAD110739068800727
:10383000C00FFBD00020596400E0401C91680906CD
:10384000C90FFAD1D864AC62AC6162B670BD000039
:1038500000040048003800401813002010B50C4642
:103860000A4601460348FFF777FF00F097FC204621
:1038700010BD00006802002010B50C460A46014643
:103880000348FFF769FF00F089FC204610BD0000E7
:103890006802002010B50C4600F0EAFC204610BD7E
:1038A00004494968F0221140034A0909515CC840A3
:1038B00070470000001002400553000803494968A2
:1038C000034A4905490F515CC84070470010024047
:1038D0001553000810B5064841680C200140054802
:1038E00005D0042903D0082901D100F005F810BD46
:1038F0000010024000127A0010B50C4C61680122E1
:1039000012040B48114002D0914200D14000E16AFC
:103910000907090F491CFCF7E7FB61680F229204B5
:103920001140890C891C484310BD00000010024062
:1039300000093D0000B50820FDF710FDC0B200BD34
:1039400070B5D417A40F0023A418A51003E09C00A1
:103950000E5906515B1C9D42F9DCD40F6B00A41874
:10396000651003E05C000E5B06535B1C9D42F9DCB6
:10397000104670BD00B5FFF7DDFF00BDF8B5134A76
:103980000024E443002117881646844625468036E5
:103990000F48874208D1708C0E4B984204D153884F
:1039A000AB4201DD0C461D46491C0829F0DB082C02
:1039B00007D2A4204443A11802466046FFF7C0FF87
:1039C00002E06046FEF732FE0020F8BD00A00008CD
:1039D000AA550000A55A00000B0702881B0F012101
:1039E00099408A430280704710B5402802DB0020CE
:1039F000C04310BD0C4BC200D218148FA40611D4C2
:103A00004000C0180D239B01C31899820B2300218D
:103A10009B01C0188182054800685063108F2021E7
:103A200008431087002010BD980A002000010020E4
:103A300010B500F001F810BD03488168C907C90F2F
:103A400000D0C068704700000030014070B51A4CCB
:103A50006168491C616019490180A1884180184949
:103A6000CA6E8280496F8160112181831549C183AB
:103A7000A1684A011449511800250B462A469E5C4C
:103A8000FF2E04D1521C202AF9D3002D10D0202261
:103A9000FCF7A4FDA0682060401CA060400101214B
:103AA00089022030884201D90020A060002070BD2A
:103AB000202200F06DFCEDE7A0000020AA550000D8
:103AC00098120020A55A000000A8000810B514465E
:103AD0000A46012802D0022806D00EE021461046F0
:103AE000FFF7CAFE064804E021461046FFF7D2FE63
:103AF000044880304168491C4160204610BD0000E8
:103B000004020020A40200200B0702881B0F0121E1
:103B100099400A43028070470907090F01238B402F
:103B20000188002A01D0194300E0994301807047C1
:103B30000907090F01238B400188002A01D019438E
:103B400000E099430180704770B50B051B0E204CB7
:103B50005B000D071C192D0F030000F053FC090634
:103B60000B14191E23282D313600FF292DD88D2046
:103B7000800003E0FF2928D89520800020182946DE
:103B8000FFF7D6FF21E0FF291FD89D208000F5E731
:103B900080291AD2F5208000F0E7802915D2FD2077
:103BA0008000EBE7402910D2A5208000E6E74029FD
:103BB0000BD2AD208000E1E7802906D20548DDE781
:103BC000802902D203482030D8E7002070BD0000D1
:103BD000980A00201404000001218903034A0028E8
:103BE00001D0916270479161704700000008004861
:103BF00001210922C902D206002801D09161704733
:103C00009162704701214903034A002801D0916263
:103C1000704791617047000000080048F8B5344CC7
:103C20004B001C1911239B01E318009321239B01D6
:103C3000E51892B28A283ED010DC2D4F2D4E4B0055
:103C4000DB199F190F26B6019E198338030000F077
:103C5000D9FB07141B1F23272B2E4C00992842D079
:103C600006DC8B282ED08C2833D08D283DD136E031
:103C7000A12838D0FE2838D135E0102935DAFF34B4
:103C8000FF340234A28630E010292EDABA822CE00A
:103C900010292ADABA8628E0082926DAB28224E036
:103CA000082922DAB28620E0FF291EDC19E0FF296C
:103CB0001BDCAA8219E0802917DA01208002201873
:103CC000828612E0402910DA0D20800105E0828210
:103CD0000BE0402909DA0B2080012018F7E7402982
:103CE00003DA0098F3E78029E3DB0020F8BD000049
:103CF000980A002040020000F0B58DB0002500F0C9
:103D0000DDFDFCF72BFE059010213A4800F038FE4F
:103D10000790FCF723FE04901021364800F0DAFDEE
:103D20000690FCF71BFE03901021324800F0F0FDD6
:103D30000190FCF713FE064610212E4800F000FE0D
:103D40000090FCF70BFE2C4A0446906801210843C2
:103D50009060881E106129481061264B0021585C34
:103D60001070491C1029FADB1768FCF7F7FD0B905F
:103D70000199009802970190214F0091781921A193
:103D8000069B079A00F02AFB45190B98A11B001B04
:103D900001910290039A04990398B21A431A00926F
:103DA00008460599421A781920A100F017FB44191A
:103DB00008A8FEF731FB26484268012000040240B3
:103DC0003819134623A100F009FB0419381926A15C
:103DD000089A00F003FB01193846FFF73FFD012167
:103DE0000D20FEF75BFC24490320886000200DB005
:103DF000F0BD0000054E00080030024001A00000A8
:103E0000040100200D0A435243202025303458205D
:103E100020253034582020253034582020253034B7
:103E2000582020253034580D0A00000074696D6553
:103E3000202530346420202530346420202530347F
:103E4000642020253034642020253034640D0A009D
:103E5000001002404D61696E536F757263652025D5
:103E600078202564200D0A00737973636C6B20251C
:103E700064200D0A000000000000002030B5002181
:103E8000114D01220846920269602B18401C1972DC
:103E90009042FADB002009220C4C920143001B19CE
:103EA0009B18401C99861028F8DB002011229201F3
:103EB00043001B199B18401C9982FF28F8DD012044
:103EC0002860002030BD000024170020980A002040
:103ED000402802DB0020C04370470B4AC10089180C
:103EE0000B8F9B060DD5400080180B2200239201FA
:103EF00080188382054800684863088F2022904319
:103F00000887002070470000980A00200001002068
:103F100010B5FCF7F7FDFCF7E5FF10BD70B594B0E8
:103F200030216846FCF75AF9002401250E94280434
:103F30000990009505200F94C0040D940226019568
:103F40000A900C9408960B956846FDF75DF80028DA
:103F500003D0862115A000F03FFA07200C900E94A4
:103F600001210D960F940CA8FCF792FE002803D0B7
:103F700092210EA000F030FA109510A81295FCF7CF
:103F800011FE002803D0A12108A000F025FA4B2043
:103F90008001FCF78FFF0420FCF754FF002211463C
:103FA000501EFCF7FBFD14B070BD00002E2E5C4BC4
:103FB0004C696E6B5C5372635C4253502E6300001D
:103FC000134801680122114301604168114A114000
:103FD00041600168104A11400160016801229204A9
:103FE0009143016041683F22120491434160C16ADC
:103FF00009090901C162016BFF2214329143016377
:10400000416B49084900416300218160704700000D
:10401000001002400CB8FF08FFFFF6FE04480169DB
:10402000C907C90F02D00121C943016170470000CF
:104030000010004070B51B4CE0691B498006C00FA2
:1040400011D01A4A01201060194A1060C869401C3A
:10405000C861A28C4868401C4860174B154D186811
:104060002A54401C1860E0690007C00F04D00820E3
:104070002062886A401C88622068C006C00F07D092
:10408000E069C006C00F03D01020206200F03CF8A9
:10409000E0694006C00F03D04020206200F076F8AF
:1040A00070BD0000003801400402002048000020DC
:1040B0004C000020440300204000002010B5104CAC
:1040C000E069E0690007C00F05D0082020620D48B4
:1040D000816A491C81622068C006C00F07D0E06970
:1040E000C006C00F03D01020206200F09FF8E069E6
:1040F0004006C00F03D04020206200F0E9F810BD58
:1041000000440040A40200200648016B491C0163E2
:1041100005480068002803DD0248012180308160E5
:10412000704700000402002040000020F8B5144D44
:104130000C46064602212846FEF786F8102000901D
:10414000104B324602212846FEF768F8224602212B
:104150002846FEF7ABF802212846FEF781F80A4808
:10416000C4630121C16002212846FEF785F8054895
:10417000283881688022114381602046F8BD000004
:104180000000024028380140040200200248C16AB1
:10419000491CC162704700000402002010B50A48A3
:1041A000C06800280DD1084CE06F6434002808D1A5
:1041B0002046FCF723FB0146E26820688018FFF7E1
:1041C000B5FF002010BD000004020020F8B5144D1A
:1041D0000C46064605212846FEF736F800200090DA
:1041E0003346104A05212846FEF718F822460521D5
:1041F0002846FEF75BF805212846FEF731F80A4805
:1042000004640121016105212846FEF735F80548BF
:10421000243881684022114381600020F8BD0000ED
:104220000000024024440040A40200200B480C4936
:1042300000794058802180B2081A0A49012208609A
:1042400009498A6080390A6B521C0A63002803DD21
:10425000012006490007486070470000164E00081C
:1042600004000240440000202403002000ED00E090
:10427000F8B5144D0C46064604212846FDF7E4FF28
:1042800010200090104B324604212846FDF7C6FF4F
:10429000224604212846FEF709F804212846FDF7A6
:1042A000DFFF0A48C4630121C16004212846FDF7ED
:1042B000E3FF054828388168802211438160204649
:1042C000F8BD00000000024028440040A402002085
:1042D0000248C16A491CC16270470000A402002064
:1042E00010B50A460249FCF779F9002010BD00001C
:1042F000007C000870B50C460B494118002B08D013
:104300000A4D4519012B03D0094B9B8A002B00D184
:1043100029460028204603D000F03AF8002070BD5E
:10432000FCF75CF9FAE700000080000800A0000834
:10433000EC140020F8B541880025491CED4380238A
:10434000418000221146114C002659430C19314678
:1043500003E0675CFF2F04D1491C9942F9DB002E72
:1043600003D0521C082AEDDB00E01546082D06D2CA
:1043700006495D436918042200F00AF803E00422AC
:104380000249FCF72BF90020F8BD000000A000084E
:10439000F7B50D460646FCF79DFB029800248708FA
:1043A00007E0A0003258411900230220FCF754FB1B
:1043B000641CA742F5D802987C00470807E060001B
:1043C000325A411900230120FCF746FB641CA74226
:1043D000F5D8FCF737FBFEBDFEE700000FB410B5C3
:1043E00004A9074B02AA039800F028F8044602A982
:1043F000002000F05DFA204610BC08BC04B018474D
:10440000B148000830B47446641E2578641CAB4281
:1044100000D21D46635D5B00E31830BC184702E024
:1044200008C8121F08C1002AFAD17047704700203F
:1044300001E001C1121F002AFBD17047FFB591B006
:104440000F460546002606E025280AD0149A13993F
:1044500090476D1C761C28780028F5D1304615B0A1
:10446000F0BD002400940121F34A029400E00443CB
:104470006D1C2B780846203B98401042F7D12878D5
:104480002A280ED0022128780246303A092A15D867
:10449000009A0A235A43303A80180C436D1C00904E
:1044A000F1E701CF0090002805DA01204003044322
:1044B000009840420090022004436D1C28782E286A
:1044C00015D10420044368786D1C2A280AD101CF35
:1044D0006D1C02900BE002990A22514330394018BA
:1044E0006D1C02902878014630390929F3D92878C3
:1044F0006C2810D006DC4C281AD068280ED06A2808
:1045000017D104E0742813D07A2812D110E00120CA
:10451000400504430CE00121090501E003210905E0
:104520000C436978814203D10120000524186D1CD9
:104530006D1C287803906E281ED00CDC632831D0C7
:1045400004DC00288AD0582811D1B2E064287BD03E
:1045500069280CD178E073282DD004DC6F2870D046
:10456000702804D1A7E075286CD078286BD0149AF5
:1045700013999047761C62E06002400F022807D032
:1045800003280AD0042838680AD006603F1D56E088
:104590003868F11706604160F8E738680680F5E78B
:1045A0000670F3E73878694608740020487404A858
:1045B0000390012003E0386803900020C0433F1DB2
:1045C00061070FD5002101E00199491C029A019170
:1045D000914213DA8142F7DB019A0399895C002941
:1045E000F2D10BE0002101E00199491C01918142C7
:1045F000FADB019A0399895C0029F5D101990098A9
:10460000139A401A00902146149B00F03BF901993F
:104610008019461807E0039803990078491C039114
:10462000149A139990470198401E0190401CF2D1B2
:104630002146149B139A009800F014F986196D1CFA
:1046400009E741E033E034E00A20002104900591BD
:104650006002410F022905D001CFC21794460329F9
:1046600005D007E0FF1DFF08FF0003CF06E000B202
:10467000C2179446042902D140B2C1178C460022C9
:104680006146944506DA0A460021404291418C4633
:104690002D2102E0210504D52B216A461176012146
:1046A00003E0E10701D02021F7E7019154E00A205F
:1046B0000BE0102009E010200490002104200443A6
:1046C00008200591029003E0082000210591049044
:1046D0006002410F022905D001CF00229446032930
:1046E00006D006E0FF1DFF08FF0003CF8C4603E065
:1046F00080B2042900D1C0B20021019121072BD53D
:104700000399702906D0049A1021059B4A401A4348
:1047100005D00EE040216A461176012108E061468D
:10472000014306D030216A46117603995176022161
:104730000191049A0821059B4A401A430CD1614615
:10474000014301D1610707D530216A461176012165
:1047500001910299491E02910399582904D037A169
:1047600003910FA90F910DE039A1F9E76146059B6F
:10477000049AFBF748FD039B8C469B5C0F9A521EE4
:104780000F92137061460143F0D10F9807A9081AE0
:1047900020300390600704D5012000048443029870
:1047A00001E0012002900399884201DD401A00E0F7
:1047B000002041180290019809180098401A0090B2
:1047C000E00306D42146149B139A009800F05AF88F
:1047D00086190020049008E006A9085C149A139931
:1047E00090470498401C761C049001998842F3DBA2
:1047F000E0030CD52146149B139A009800F042F870
:10480000861904E0149A302013999047761C029977
:10481000481E02900029F5DC08E00F980F990078F7
:10482000491C0F91149A13999047761C0399481EBE
:1048300003900029F1DCFBE6092801003031323316
:1048400034353637383961626364656600000000CC
:1048500030313233343536373839414243444546B6
:1048600000000000F8B5044600251E4617468804DF
:1048700004D405E039462020B0476D1C641EF9D5EC
:104880002846F8BDFFB50446002581B01E46C80382
:1048900001D5302700E02027880404D505E03846FC
:1048A0000399B0476D1C641EF9D5284605B0F0BDCC
:1048B0000A68531C0B6010707047000010B50A2185
:1048C00001A0FEF7CBFF10BD1B5B324A1B5B303BE8
:1048D0003048000030B503460B48002900D10121C3
:1048E0000A4C491E0ED31A7850400022C50702D048
:1048F0004008604000E04008521CD2B2082AF5D3BC
:104900005B1CEEE730BD0000FFFF000001A00000CF
:1049100070B50A4DFF23EE1D1A46F93605E00478FE
:1049200054402A5D5A40335D401C0C46491E89B2F2
:10493000002CF4D11802104370BD00001C50000878
:1049400070B504460C4800220C4E11E02378521C2E
:104950001D4645402D07ED0E755B000945401809C1
:1049600068400007C00E305A2B09584092B2641CB0
:104970008A42EBD370BD0000FFFF0000E052000848
:1049800010B5084A084B07E0047854402406E40DAB
:104990001C5B120A6240401C491EF5D2D04380B213
:1049A00010BD0000FFFF00001C4E000810B572B6DD
:1049B00004210A4A916149030C11022393620842BF
:1049C00001D0946100E094624908022393610029B8
:1049D000F3D104209062906162B610BD00040048DB
:1049E00006C00021016041608160C1600122026156
:1049F00041610846704700001FB5FF201930D74BB2
:104A0000FF22009001321946D548FCF7B9FA802000
:104A1000D44B024600901946D348FCF7B1FAFCF794
:104A200079F80021D14A0F4660204843801847603A
:104A30008760076147618761C76107628762476274
:104A4000C762491C07630929EEDBC94DC9482F61BC
:104A5000C06A6860C8480068A860C848406AE860E2
:104A6000FFF75CFAC749C6480860FCF799FAFDF7FA
:104A70008DFEFDF777FEFDF747FBC348FEF77EFF8F
:104A8000FEF778FF2C46803C4207C049520F606514
:104A90000A700121BE4E0F2805D0000706D5BD487B
:104AA0000170377005E0BC480170F8E7B94807703D
:104AB0003170BA48BA49027001200870E120B94942
:104AC00080020860FDF7C4FFFEF754F8FDF7DCFE36
:104AD000B548426840210A434260FDF735FFFDF7C3
:104AE000EFFDFDF7B7FEFDF789FFB0480168012231
:104AF00011430160AE480168202211430160016842
:104B0000102211430160016840221143016080219D
:104B1000A848FFF75BFBA848016810221143016019
:104B200001684022114301600A20FBF72DFF01209C
:104B3000FFF768F80020FFF74FF80020FCF75BFA5A
:104B40000120FBF735FD9D48FFF730FF0120FBF703
:104B500039FD0020FFF74CF8FFF7CEF8FBF7FEFE1B
:104B6000686097480782008A012803D1FCF7C0F9E2
:104B7000FFF784F993485A210290418078488030A9
:104B800001909048403803908F4E0120377070702C
:104B9000FBF7E4FEF060FBF7AFFF0090E065FBF78A
:104BA00065FE039980B28886FFF700FFFBF7D6FE0B
:104BB0003061206EC006C00E022818D1FBF776FBCC
:104BC00082480168002982490A680AD0002A0ED169
:104BD000006808607F4800687F490860FEF79CFA1B
:104BE00005E0002A03D000680860FEF7AFFA7448B9
:104BF000018A01290ED16749097800290AD0818AE2
:104C0000002928D075497160C18A754801607068B3
:104C1000FEF7A4FA686831696960081AA860E96853
:104C2000884200D2E8602969884200D92861FBF7F0
:104C300095FE706157480078002806D057480078E4
:104C4000002802D00220FCF767FC0098800404D5FD
:104C50000120307002E06349D5E737700098000505
:104C600002D50120707000E0777049480078002874
:104C70001AD00220FCF730FE606E002801D15A489D
:104C80000770594801780298818258490868800461
:104C900002D50120307000E037700868000502D5A9
:104CA0000120707000E07770606E002801D0401E17
:104CB0006066A06E002801D0401EA066606E0028CD
:104CC00045D07078FEF79EFFA06E002841D0707826
:104CD000FEF782FF0020FEF78BFFFBF73FFEB0617F
:104CE0000298808AFCF787F9FBF738FEF061FBF742
:104CF00035FE0A2130620846FBF7E6F90020401C29
:104D00004028FCDB206E3A4E401C206630680028AC
:104D100012DD0199896800290ED082B2354901203F
:104D2000FDF7F0FF002804D0324901203268FCF77B
:104D3000F9FE37600198876015480078002802D096
:104D40000020FBF721FE2D492B4808601CE7307836
:104D5000B8E70020FEF740FF0120BCE70C1500205B
:104D60000402002024160020A40200206405002074
:104D70001813002080F7FF1F3400002000100240AD
:104D80001027000018000020F40900205A0000201D
:104D900059000020580000209000002061000020F1
:104DA0005B0000203800002000300140001000406F
:104DB00000380140C403002000440040FFFF000011
:104DC000EC140020D80C0020D0000020C4000020EB
:104DD000C80000201C000020CC00002000A000081B
:104DE000F800002000800008440400207400002027
:104DF0004000002044030020AAAA00000030004028
:104E0000081C304458112233445566778899AABB50
:104E1000CCDDEEFF0000081C304458000000891172
:104E200012239B322446AD573665BF74488CC19D12
:104E30005AAFD3BE6CCAE5DB7EE9F7F881100801F2
:104E400093331A22A5562C47B7753E64C99C408DF2
:104E5000DBBF52AEEDDA64CBFFF976E802218B308E
:104E6000100299132667AF763444BD554AADC3BCD2
:104E7000588ED19F6EEBE7FA7CC8F5D983310A20B2
:104E800091121803A7772E66B5543C45CBBD42ACB2
:104E9000D99E508FEFFB66EAFDD874C904428D534A
:104EA00016619F702004A9153227BB364CCEC5DF92
:104EB0005EEDD7FC6888E1997AABF3BA85520C4372
:104EC00097711E60A1142805B3373A26CDDE44CF72
:104ED000DFFD56ECE9986089FBBB72AA06638F720E
:104EE00014409D512225AB343006B9174EEFC7FE52
:104EF0005CCCD5DD6AA9E3B8788AF19B87730E6232
:104F000095501C41A3352A24B1163807CFFF46EE31
:104F1000DDDC54CDEBB962A8F99A708B08848195D9
:104F20001AA793B62CC2A5D33EE1B7F04008C91921
:104F3000522BDB3A644EED5F766DFF7C89940085E1
:104F40009BB712A6ADD224C3BFF136E0C118480901
:104F5000D33B5A2AE55E6C4FF77D7E6C0AA583B47D
:104F6000188691972EE3A7F23CC0B5D14229CB38E1
:104F7000500AD91B666FEF7E744CFD5D8BB502A4A1
:104F800099961087AFF326E2BDD034C1C3394A28C1
:104F9000D11A580BE77F6E6EF55C7C4D0CC685D739
:104FA0001EE597F42880A1913AA3B3B2444ACD5BA1
:104FB0005669DF78600CE91D722FFB3E8DD604C761
:104FC0009FF516E4A9902081BBB332A2C55A4C4B81
:104FD000D7795E68E11C680DF33F7A2E0EE787F6FD
:104FE0001CC495D52AA1A3B03882B193466BCF7A61
:104FF0005448DD59622DEB3C700EF91F8FF706E621
:105000009DD414C5ABB122A0B9923083C77B4E6A40
:10501000D5585C49E33D6A2CF11E780F00C18140F0
:1050200001C0804101C0804100C1814001C0804178
:1050300000C1814000C1814001C0804101C0804168
:1050400000C1814000C1814001C0804100C1814058
:1050500001C0804101C0804100C1814001C0804148
:1050600000C1814000C1814001C0804100C1814038
:1050700001C0804101C0804100C1814000C1814028
:1050800001C0804101C0804100C1814001C0804118
:1050900000C1814000C1814001C0804101C0804108
:1050A00000C1814000C1814001C0804100C18140F8
:1050B00001C0804101C0804100C1814000C18140E8
:1050C00001C0804101C0804100C1814001C08041D8
:1050D00000C1814000C1814001C0804100C18140C8
:1050E00001C0804101C0804100C1814001C08041B8
:1050F00000C1814000C1814001C0804101C08041A8
:1051000000C1814000C1814001C0804100C1814097
:1051100001C0804101C0804100C1814000C0C10187
:10512000C30302C2C60607C705C5C404CC0C0DCD17
:105130000FCFCE0E0ACACB0BC90908C8D81819D987
:105140001BDBDA1A1EDEDF1FDD1D1CDC14D4D515B7
:10515000D71716D6D21213D311D1D010F03031F1A7
:1051600033F3F23236F6F737F53534F43CFCFD3DD7
:10517000FF3F3EFEFA3A3BFB39F9F83828E8E929C7
:10518000EB2B2AEAEE2E2FEF2DEDEC2CE42425E577
:1051900027E7E62622E2E323E12120E0A06061A1E7
:1051A00063A3A26266A6A767A56564A46CACAD6D97
:1051B000AF6F6EAEAA6A6BAB69A9A86878B8B97907
:1051C000BB7B7ABABE7E7FBF7DBDBC7CB47475B537
:1051D00077B7B67672B2B373B17170B05090915127
:1051E0009353529296565797559594549C5C5D9D57
:1051F0005F9F9E5E5A9A9B5B995958988848498947
:105200004B8B8A4A4E8E8F4F8D4D4C8C44848545F6
:1052100087474686824243834181804009000001DE
:10522000000100011010000000000000AA5500005D
:10523000000100000000000000000000000000006D
:10524000000001000000000906000000000000004E
:10525000010000000009070000000000000000003D
:10526000000000000000000000000000000010101E
:10527000101010101010101010101010101000004E
:10528000030000000400000005000000060000000C
:105290000700000008000000090000000A000000EC
:1052A0000B0000000C0000000D0000000E000000CC
:1052B0000F000000100000000000000000000000CF
:1052C0000000000000000000000000001100A55ACE
:1052D000AA550000000000000000000000000000CF
:1052E000000001CC01D8001401F0003C002801E4CA
:1052F00001A0006C007801B40050019C01880044BA
:10530000081C3044580000000000000000010203A7
:105310000406070809000000000102030400000061
:105320004053000800000020040100001E44000853
:1053300044540008040100204C1C00002E440008C6
:10534000000000000000000000000000000000005D
:105350000000000001000000102700000000000015
:10536000000000000000000000000000000000003D
:1053700000000000000000000084030040420F0015
:10538000000000000000000000000000000000001D
:10539000000000000000000000000000000101010A
:1053A00000000000000000000000000000000000FD
:1053B00000000000000000000000000000000000ED
:1053C00000000000000000000000000000000000DD
:1053D00000000000010000000000000000000000CC
:1053E000FFFFFFFF000000000000000000000000C1
:1053F00000000000000000000000000000000000AD
:10540000000000000000000000000000000000009C
:105410000000000000800008000000000000000004
:10542000000000000000000000000000000000007C
:10543000000000000100000097000000001BB70002
:045440000000000068
:04000005080000B53A
:00000001FF
